 rndc

 Timestamp is 407b876a (Tue Apr 13 16:23:38 2004)

 Preferred load address is 00400000

 Start         Length     Name                   Class
 0001:00000000 00007c14H .text                   CODE
 0002:00000000 00000f24H .rdata                  DATA
 0002:00000f24 00000004H .rtc$IAA                DATA
 0002:00000f28 00000004H .rtc$IZZ                DATA
 0002:00000f2c 00000004H .rtc$TAA                DATA
 0002:00000f30 00000004H .rtc$TZZ                DATA
 0002:00000f34 00000000H .edata                  DATA
 0003:00000000 00000004H .CRT$XCA                DATA
 0003:00000004 00000004H .CRT$XCAA               DATA
 0003:00000008 00000004H .CRT$XCZ                DATA
 0003:0000000c 00000004H .CRT$XIA                DATA
 0003:00000010 0000000cH .CRT$XIC                DATA
 0003:0000001c 00000004H .CRT$XIZ                DATA
 0003:00000020 00000004H .CRT$XPA                DATA
 0003:00000024 00000004H .CRT$XPX                DATA
 0003:00000028 00000004H .CRT$XPZ                DATA
 0003:0000002c 00000004H .CRT$XTA                DATA
 0003:00000030 00000004H .CRT$XTZ                DATA
 0003:00000040 00001ce0H .data                   DATA
 0003:00001d20 00002764H .bss                    DATA
 0004:00000000 00000064H .idata$2                DATA
 0004:00000064 00000014H .idata$3                DATA
 0004:00000078 00000234H .idata$4                DATA
 0004:000002ac 00000234H .idata$5                DATA
 0004:000004e0 00000a80H .idata$6                DATA

  Address         Publics by Value              Rva+Base     Lib:Object

 0000:00000000       __except_list              00000000     <absolute>
 0001:00000000       _main                      00401000 f   rndc.obj
 0001:000017f7       _notify                    004027f7 f   util.obj
 0001:00001834       _fatal                     00402834 f   util.obj
 0001:00001888       _isc_mem_destroy           00402888 f   libisc:libisc.dll
 0001:0000188e       _isc_mem_stats             0040288e f   libisc:libisc.dll
 0001:00001894       _isc__mem_put              00402894 f   libisc:libisc.dll
 0001:0000189a       _isc_log_destroy           0040289a f   libisc:libisc.dll
 0001:000018a0       _isc_socketmgr_destroy     004028a0 f   libisc:libisc.dll
 0001:000018a6       _isc_taskmgr_destroy       004028a6 f   libisc:libisc.dll
 0001:000018ac       _isc_task_detach           004028ac f   libisc:libisc.dll
 0001:000018b2       _isc_socket_cancel         004028b2 f   libisc:libisc.dll
 0001:000018b8       _isc_app_run               004028b8 f   libisc:libisc.dll
 0001:000018be       _isc_app_onrun             004028be f   libisc:libisc.dll
 0001:000018c4       _isc__mem_get              004028c4 f   libisc:libisc.dll
 0001:000018ca       _isc_log_usechannel        004028ca f   libisc:libisc.dll
 0001:000018d0       _isc_log_createchannel     004028d0 f   libisc:libisc.dll
 0001:000018d6       _isc_log_settag            004028d6 f   libisc:libisc.dll
 0001:000018dc       _isc_log_setcontext        004028dc f   libisc:libisc.dll
 0001:000018e2       _isc_log_create            004028e2 f   libisc:libisc.dll
 0001:000018e8       _isc_task_create           004028e8 f   libisc:libisc.dll
 0001:000018ee       _isc_taskmgr_create        004028ee f   libisc:libisc.dll
 0001:000018f4       _isc_socketmgr_create      004028f4 f   libisc:libisc.dll
 0001:000018fa       _isc_mem_create            004028fa f   libisc:libisc.dll
 0001:00001900       _isc_random_get            00402900 f   libisc:libisc.dll
 0001:00001906       _isc_commandline_parse     00402906 f   libisc:libisc.dll
 0001:0000190c       _isc_result_totext         0040290c f   libisc:libisc.dll
 0001:00001912       _isc_app_start             00402912 f   libisc:libisc.dll
 0001:00001918       _isc_ntpaths_get           00402918 f   libisc:libisc.dll
 0001:0000191e       _isc_file_progname         0040291e f   libisc:libisc.dll
 0001:00001924       _isc_event_free            00402924 f   libisc:libisc.dll
 0001:0000192a       _isc_app_unblock           0040292a f   libisc:libisc.dll
 0001:00001930       _isc_app_block             00402930 f   libisc:libisc.dll
 0001:00001936       _isc_socket_connect        00402936 f   libisc:libisc.dll
 0001:0000193c       _isc_socket_create         0040293c f   libisc:libisc.dll
 0001:00001942       _isc_sockaddr_pf           00402942 f   libisc:libisc.dll
 0001:00001948       _isc_sockaddr_format       00402948 f   libisc:libisc.dll
 0001:0000194e       _isc_socket_send           0040294e f   libisc:libisc.dll
 0001:00001954       _isc__buffer_putuint32     00402954 f   libisc:libisc.dll
 0001:0000195a       _isc__buffer_init          0040295a f   libisc:libisc.dll
 0001:00001960       _isc_stdtime_get           00402960 f   libisc:libisc.dll
 0001:00001966       _isc_socket_detach         00402966 f   libisc:libisc.dll
 0001:0000196c       _isc_error_runtimecheck    0040296c f   libisc:libisc.dll
 0001:00001972       _isc_app_shutdown          00402972 f   libisc:libisc.dll
 0001:00001978       _isc_task_shutdown         00402978 f   libisc:libisc.dll
 0001:0000197e       _isc_file_exists           0040297e f   libisc:libisc.dll
 0001:00001984       _cfg_parser_destroy        00402984 f   libisccfg:libisccfg.dll
 0001:0000198a       _cfg_obj_destroy           0040298a f   libisccfg:libisccfg.dll
 0001:00001990       _cfg_obj_asuint32          00402990 f   libisccfg:libisccfg.dll
 0001:00001996       _cfg_map_getname           00402996 f   libisccfg:libisccfg.dll
 0001:0000199c       _cfg_listelt_value         0040299c f   libisccfg:libisccfg.dll
 0001:000019a2       _cfg_list_next             004029a2 f   libisccfg:libisccfg.dll
 0001:000019a8       _cfg_list_first            004029a8 f   libisccfg:libisccfg.dll
 0001:000019ae       _cfg_obj_asstring          004029ae f   libisccfg:libisccfg.dll
 0001:000019b4       _cfg_map_get               004029b4 f   libisccfg:libisccfg.dll
 0001:000019ba       _cfg_parse_file            004029ba f   libisccfg:libisccfg.dll
 0001:000019c0       _cfg_parser_create         004029c0 f   libisccfg:libisccfg.dll
 0001:000019c6       _isccc_ccmsg_invalidate    004029c6 f   libisccc:libisccc.dll
 0001:000019cc       _isccc_result_register     004029cc f   libisccc:libisccc.dll
 0001:000019d2       _isccc_ccmsg_readmessage   004029d2 f   libisccc:libisccc.dll
 0001:000019d8       _isccc_ccmsg_setmaxsize    004029d8 f   libisccc:libisccc.dll
 0001:000019de       _isccc_ccmsg_init          004029de f   libisccc:libisccc.dll
 0001:000019e4       _isccc_cc_towire           004029e4 f   libisccc:libisccc.dll
 0001:000019ea       _isccc_cc_definestring     004029ea f   libisccc:libisccc.dll
 0001:000019f0       _isccc_alist_lookup        004029f0 f   libisccc:libisccc.dll
 0001:000019f6       _isccc_cc_createmessage    004029f6 f   libisccc:libisccc.dll
 0001:000019fc       _isccc_sexpr_free          004029fc f   libisccc:libisccc.dll
 0001:00001a02       _isccc_ccmsg_cancelread    00402a02 f   libisccc:libisccc.dll
 0001:00001a08       _isccc_cc_defineuint32     00402a08 f   libisccc:libisccc.dll
 0001:00001a0e       _isccc_cc_lookupuint32     00402a0e f   libisccc:libisccc.dll
 0001:00001a14       _isccc_cc_fromwire         00402a14 f   libisccc:libisccc.dll
 0001:00001a1a       _isccc_cc_lookupstring     00402a1a f   libisccc:libisccc.dll
 0001:00001a20       _isccc_base64_decode       00402a20 f   libisccc:libisccc.dll
 0001:00001a26       _bind9_getaddresses        00402a26 f   libbind9:libbind9.dll
 0001:00001a30       _strcmp                    00402a30 f   LIBCMT:strcmp.obj
 0001:00001ac0       _strlen                    00402ac0 f   LIBCMT:strlen.obj
 0001:00001b4b       ___initstdio               00402b4b f   LIBCMT:_file.obj
 0001:00001bf4       ___endstdio                00402bf4 f   LIBCMT:_file.obj
 0001:00001c08       __lock_file                00402c08 f   LIBCMT:_file.obj
 0001:00001c37       __lock_file2               00402c37 f   LIBCMT:_file.obj
 0001:00001c5a       __unlock_file              00402c5a f   LIBCMT:_file.obj
 0001:00001c89       __unlock_file2             00402c89 f   LIBCMT:_file.obj
 0001:00001cac       _atol                      00402cac f   LIBCMT:atox.obj
 0001:00001d34       _atoi                      00402d34 f   LIBCMT:atox.obj
 0001:00001d40       _memcpy                    00402d40 f   LIBCMT:memcpy.obj
 0001:0000207d       ___crtExitProcess          0040307d f   LIBCMT:crt0dat.obj
 0001:000020ad       __lockexit                 004030ad f   LIBCMT:crt0dat.obj
 0001:000020b6       __unlockexit               004030b6 f   LIBCMT:crt0dat.obj
 0001:000020bf       __cinit                    004030bf f   LIBCMT:crt0dat.obj
 0001:000021f7       _exit                      004031f7 f   LIBCMT:crt0dat.obj
 0001:00002208       __exit                     00403208 f   LIBCMT:crt0dat.obj
 0001:00002219       __cexit                    00403219 f   LIBCMT:crt0dat.obj
 0001:00002228       __c_exit                   00403228 f   LIBCMT:crt0dat.obj
 0001:00002237       _fprintf                   00403237 f   LIBCMT:fprintf.obj
 0001:00002295       _printf                    00403295 f   LIBCMT:printf.obj
 0001:000022fb       __stricmp                  004032fb f   LIBCMT:stricmp.obj
 0001:00002364       _fputs                     00403364 f   LIBCMT:fputs.obj
 0001:000023d5       _vfprintf                  004033d5 f   LIBCMT:vfprintf.obj
 0001:00002432       __amsg_exit                00403432 f   LIBCMT:crt0.obj
 0001:0000247b       _mainCRTStartup            0040347b f   LIBCMT:crt0.obj
 0001:00002638       __ioinit                   00403638 f   LIBCMT:ioinit.obj
 0001:00002836       _calloc                    00403836 f   LIBCMT:calloc.obj
 0001:000028f1       __fcloseall                004038f1 f   LIBCMT:closeall.obj
 0001:0000298c       __flush                    0040398c f   LIBCMT:fflush.obj
 0001:000029e9       __fflush_lk                004039e9 f   LIBCMT:fflush.obj
 0001:00002aec       __flushall                 00403aec f   LIBCMT:fflush.obj
 0001:00002af5       __mtinitlocks              00403af5 f   LIBCMT:mlock.obj
 0001:00002b3e       __mtdeletelocks            00403b3e f   LIBCMT:mlock.obj
 0001:00002b93       __unlock                   00403b93 f   LIBCMT:mlock.obj
 0001:00002ba8       __mtinitlocknum            00403ba8 f   LIBCMT:mlock.obj
 0001:00002c27       __lock                     00403c27 f   LIBCMT:mlock.obj
 0001:00002c58       ___isctype_mt              00403c58 f   LIBCMT:isctype.obj
 0001:00002ccf       ___freetlocinfo            00403ccf f   LIBCMT:setlocal.obj
 0001:00002e5b       ___updatetlocinfo          00403e5b f   LIBCMT:setlocal.obj
 0001:00002e96       __mtterm                   00403e96 f   LIBCMT:tidtable.obj
 0001:00002eb4       __getptd                   00403eb4 f   LIBCMT:tidtable.obj
 0001:00002f25       __mtinit                   00403f25 f   LIBCMT:tidtable.obj
 0001:00002fa0       __allmul                   00403fa0 f   LIBCMT:llmul.obj
 0001:00003054       ___onexitinit              00404054 f   LIBCMT:onexit.obj
 0001:0000307c       __onexit                   0040407c f   LIBCMT:onexit.obj
 0001:000030b4       _atexit                    004040b4 f   LIBCMT:onexit.obj
 0001:000030c6       __RTC_Initialize           004040c6 f   LIBCMT:initsect.obj
 0001:0000310a       __RTC_Terminate            0040410a f   LIBCMT:initsect.obj
 0001:0000314e       __stbuf                    0040414e f   LIBCMT:_sftbuf.obj
 0001:000031d6       __ftbuf                    004041d6 f   LIBCMT:_sftbuf.obj
 0001:0000328e       __output                   0040428e f   LIBCMT:output.obj
 0001:00003a24       __SEH_prolog               00404a24 f   LIBCMT:sehprolg.obj
 0001:00003a5f       __SEH_epilog               00404a5f f   LIBCMT:sehprolg.obj
 0001:00003a70       ___tolower_mt              00404a70 f   LIBCMT:tolower.obj
 0001:00003b40       ___ascii_stricmp           00404b40 f   LIBCMT:_stricmp.obj
 0001:00003b8e       __fwrite_lk                00404b8e f   LIBCMT:fwrite.obj
 0001:00003c95       __NMSG_WRITE               00404c95 f   LIBCMT:crt0msg.obj
 0001:00003e0c       __FF_MSGBANNER             00404e0c f   LIBCMT:crt0msg.obj
 0001:00003e45       __XcptFilter               00404e45 f   LIBCMT:winxfltr.obj
 0001:00003fa9       __setenvp                  00404fa9 f   LIBCMT:stdenvp.obj
 0001:000041dc       __setargv                  004051dc f   LIBCMT:stdargv.obj
 0001:0000427e       ___crtGetEnvironmentStringsA 0040527e f   LIBCMT:a_env.obj
 0001:000043a0       ___heap_select             004053a0 f   LIBCMT:heapinit.obj
 0001:000043ba       __heap_init                004053ba f   LIBCMT:heapinit.obj
 0001:00004410       __alloca_probe             00405410     LIBCMT:chkstk.obj
 0001:00004410       __chkstk                   00405410 f   LIBCMT:chkstk.obj
 0001:0000445d       ___crtInitCritSecAndSpinCount 0040545d f   LIBCMT:initcrit.obj
 0001:000044e8       __heap_alloc               004054e8 f   LIBCMT:malloc.obj
 0001:00004563       __nh_malloc                00405563 f   LIBCMT:malloc.obj
 0001:0000458f       _malloc                    0040558f f   LIBCMT:malloc.obj
 0001:000045a1       _free                      004055a1 f   LIBCMT:free.obj
 0001:00004612       __callnewh                 00405612 f   LIBCMT:handler.obj
 0001:00004630       _memset                    00405630 f   LIBCMT:memset.obj
 0001:00004690       ___sbh_heap_init           00405690 f   LIBCMT:sbheap.obj
 0001:000046d8       ___sbh_find_block          004056d8 f   LIBCMT:sbheap.obj
 0001:00004703       ___sbh_free_block          00405703 f   LIBCMT:sbheap.obj
 0001:00004a1b       ___sbh_alloc_new_region    00405a1b f   LIBCMT:sbheap.obj
 0001:00004ad2       ___sbh_alloc_new_group     00405ad2 f   LIBCMT:sbheap.obj
 0001:00004bd8       ___sbh_resize_block        00405bd8 f   LIBCMT:sbheap.obj
 0001:00004eb7       ___sbh_alloc_block         00405eb7 f   LIBCMT:sbheap.obj
 0001:000051b3       __fclose_lk                004061b3 f   LIBCMT:fclose.obj
 0001:000051ff       _fclose                    004061ff f   LIBCMT:fclose.obj
 0001:00005250       __write_lk                 00406250 f   LIBCMT:write.obj
 0001:000053f5       __write                    004063f5 f   LIBCMT:write.obj
 0001:000054a0       __commit                   004064a0 f   LIBCMT:commit.obj
 0001:0000555c       __errno                    0040655c f   LIBCMT:dosmap.obj
 0001:00005565       ___doserrno                00406565 f   LIBCMT:dosmap.obj
 0001:0000556e       __dosmaperr                0040656e f   LIBCMT:dosmap.obj
 0001:000055e1       ___crtGetStringTypeA       004065e1 f   LIBCMT:a_str.obj
 0001:0000579b       ___free_lc_time            0040679b f   LIBCMT:inittime.obj
 0001:0000592b       ___free_lconv_num          0040692b f   LIBCMT:initnum.obj
 0001:0000598a       ___free_lconv_mon          0040698a f   LIBCMT:initmon.obj
 0001:00005a70       _strcpy                    00406a70 f   LIBCMT:strcat.obj
 0001:00005a80       _strcat                    00406a80 f   LIBCMT:strcat.obj
 0001:00005b70       _strcspn                   00406b70 f   LIBCMT:strcspn.obj
 0001:00005bc0       _strncpy                   00406bc0 f   LIBCMT:strncpy.obj
 0001:00005d15       @__security_check_cookie@4 00406d15 f   LIBCMT:seccook.obj
 0001:00005d30       _memcmp                    00406d30 f   LIBCMT:memcmp.obj
 0001:00005df0       _strncmp                   00406df0 f   LIBCMT:strncmp.obj
 0001:00005e30       _strpbrk                   00406e30 f   LIBCMT:strpbrk.obj
 0001:00005e70       __global_unwind2           00406e70 f   LIBCMT:exsup.obj
 0001:00005eb2       __local_unwind2            00406eb2 f   LIBCMT:exsup.obj
 0001:00005f0a       __NLG_Return2              00406f0a     LIBCMT:exsup.obj
 0001:00005f1a       __abnormal_termination     00406f1a f   LIBCMT:exsup.obj
 0001:00005f3d       __NLG_Notify1              00406f3d f   LIBCMT:exsup.obj
 0001:00005f46       __NLG_Notify               00406f46 f   LIBCMT:exsup.obj
 0001:00005f59       __NLG_Dispatch             00406f59     LIBCMT:exsup.obj
 0001:000062de       __setmbcp                  004072de f   LIBCMT:mbctype.obj
 0001:0000642e       ___initmbctable            0040742e f   LIBCMT:mbctype.obj
 0001:0000644c       _realloc                   0040744c f   LIBCMT:realloc.obj
 0001:000065f9       __msize                    004075f9 f   LIBCMT:msize.obj
 0001:0000666f       __isatty                   0040766f f   LIBCMT:isatty.obj
 0001:00006699       __flsbuf                   00407699 f   LIBCMT:_flsbuf.obj
 0001:000067b2       ___wctomb_mt               004077b2 f   LIBCMT:wctomb.obj
 0001:00006812       _wctomb                    00407812 f   LIBCMT:wctomb.obj
 0001:00006840       __aulldvrm                 00407840 f   LIBCMT:ulldvrm.obj
 0001:000068e0       __except_handler3          004078e0 f   LIBCMT:exsup3.obj
 0001:0000699d       __seh_longjmp_unwind@4     0040799d f   LIBCMT:exsup3.obj
 0001:000069b8       ___crtLCMapStringA         004079b8 f   LIBCMT:a_map.obj
 0001:00006d74       ___crtMessageBoxA          00407d74 f   LIBCMT:crtmbox.obj
 0001:00006e70       _memmove                   00407e70 f   LIBCMT:memmove.obj
 0001:000071ad       __close_lk                 004081ad f   LIBCMT:close.obj
 0001:00007230       __close                    00408230 f   LIBCMT:close.obj
 0001:000072cb       __freebuf                  004082cb f   LIBCMT:_freebuf.obj
 0001:000072f6       __lseeki64_lk              004082f6 f   LIBCMT:lseeki64.obj
 0001:00007379       __free_osfhnd              00408379 f   LIBCMT:osfinfo.obj
 0001:000073f8       __get_osfhandle            004083f8 f   LIBCMT:osfinfo.obj
 0001:00007439       __lock_fhandle             00408439 f   LIBCMT:osfinfo.obj
 0001:000074ac       __unlock_fhandle           004084ac f   LIBCMT:osfinfo.obj
 0001:000074ce       ___ansicp                  004084ce f   LIBCMT:convrtcp.obj
 0001:00007517       ___convertcp               00408517 f   LIBCMT:convrtcp.obj
 0001:000076e6       __resetstkoflw             004086e6 f   LIBCMT:resetstk.obj
 0001:000077b7       ___security_init_cookie    004087b7 f   LIBCMT:seccinit.obj
 0001:0000780d       ___security_error_handler  0040880d f   LIBCMT:secfail.obj
 0001:00007957       __lseek_lk                 00408957 f   LIBCMT:lseek.obj
 0001:000079cb       __lseek                    004089cb f   LIBCMT:lseek.obj
 0001:00007a76       __getbuf                   00408a76 f   LIBCMT:_getbuf.obj
 0001:00007aba       __fptrap                   00408aba f   LIBCMT:crt0fp.obj
 0001:00007ad0       ___ascii_strnicmp          00408ad0 f   LIBCMT:_strnicm.obj
 0001:00007b50       _strchr                    00408b50 f   LIBCMT:strchr.obj
 0001:00007b56       ___from_strstr_to_strchr   00408b56     LIBCMT:strchr.obj
 0001:00007c0e       _RtlUnwind@16              00408c0e f   kernel32:KERNEL32.dll
 0002:00000000       ??_C@_01EEMJAFIK@?6?$AA@   00409000     util.obj
 0002:00000004       ??_C@_04PFAOODAA@?$CFs?3?5?$AA@ 00409004     util.obj
 0002:0000000c       ??_C@_0P@MIGLKIOC@CorExitProcess?$AA@ 0040900c     LIBCMT:crt0dat.obj
 0002:0000001c       ??_C@_0M@MBOPBNBK@mscoree?4dll?$AA@ 0040901c     LIBCMT:crt0dat.obj
 0002:00000270       ___lookuptable             00409270     LIBCMT:output.obj
 0002:000002cc       ??_C@_1O@CEDCILHN@?$AA?$CI?$AAn?$AAu?$AAl?$AAl?$AA?$CJ?$AA?$AA@ 004092cc     LIBCMT:output.obj
 0002:000002dc       ??_C@_06OJHGLDPL@?$CInull?$CJ?$AA@ 004092dc     LIBCMT:output.obj
 0002:000002e4       ??_C@_0P@GGKDKEEG@runtime?5error?5?$AA@ 004092e4     LIBCMT:crt0msg.obj
 0002:000002f4       ??_C@_02PCIJFNDE@?$AN?6?$AA@ 004092f4     LIBCMT:crt0msg.obj
 0002:000002f8       ??_C@_0O@MJNIPGOH@TLOSS?5error?$AN?6?$AA@ 004092f8     LIBCMT:crt0msg.obj
 0002:00000308       ??_C@_0N@BONNPDHF@SING?5error?$AN?6?$AA@ 00409308     LIBCMT:crt0msg.obj
 0002:00000318       ??_C@_0P@MBDAJNE@DOMAIN?5error?$AN?6?$AA@ 00409318     LIBCMT:crt0msg.obj
 0002:00000328       ??_C@_0CF@KJDAIALP@R6028?$AN?6?9?5unable?5to?5initialize?5he@ 00409328     LIBCMT:crt0msg.obj
 0002:00000350       ??_C@_0DF@GAKBPDFP@R6027?$AN?6?9?5not?5enough?5space?5for?5lo@ 00409350     LIBCMT:crt0msg.obj
 0002:00000388       ??_C@_0DF@IBLNNAIG@R6026?$AN?6?9?5not?5enough?5space?5for?5st@ 00409388     LIBCMT:crt0msg.obj
 0002:000003c0       ??_C@_0CG@IOHKGFNJ@R6025?$AN?6?9?5pure?5virtual?5function?5c@ 004093c0     LIBCMT:crt0msg.obj
 0002:000003e8       ??_C@_0DF@JIJJFJDC@R6024?$AN?6?9?5not?5enough?5space?5for?5_o@ 004093e8     LIBCMT:crt0msg.obj
 0002:00000420       ??_C@_0CJ@EGEJHFME@R6019?$AN?6?9?5unable?5to?5open?5console?5@ 00409420     LIBCMT:crt0msg.obj
 0002:0000044c       ??_C@_0CB@GNHNIELH@R6018?$AN?6?9?5unexpected?5heap?5error?$AN?6@ 0040944c     LIBCMT:crt0msg.obj
 0002:00000470       ??_C@_0CN@FOLDKNG@R6017?$AN?6?9?5unexpected?5multithread?5@ 00409470     LIBCMT:crt0msg.obj
 0002:000004a0       ??_C@_0CM@FAHFJNHO@R6016?$AN?6?9?5not?5enough?5space?5for?5th@ 004094a0     LIBCMT:crt0msg.obj
 0002:000004d0       ??_C@_0JG@LBKMGKLD@?$AN?6This?5application?5has?5requested@ 004094d0     LIBCMT:crt0msg.obj
 0002:00000568       ??_C@_0CM@FLCNIPKK@R6009?$AN?6?9?5not?5enough?5space?5for?5en@ 00409568     LIBCMT:crt0msg.obj
 0002:00000594       ??_C@_0CK@KMMJOAPP@R6008?$AN?6?9?5not?5enough?5space?5for?5ar@ 00409594     LIBCMT:crt0msg.obj
 0002:000005c0       ??_C@_0CF@HOHMHDEK@R6002?$AN?6?9?5floating?5point?5not?5load@ 004095c0     LIBCMT:crt0msg.obj
 0002:000005e8       ??_C@_0CF@GOGNBNAK@Microsoft?5Visual?5C?$CL?$CL?5Runtime?5Lib@ 004095e8     LIBCMT:crt0msg.obj
 0002:00000610       ??_C@_02PHMGELLB@?6?6?$AA@ 00409610     LIBCMT:crt0msg.obj
 0002:00000614       ??_C@_0BK@OFGJDLJJ@Runtime?5Error?$CB?6?6Program?3?5?$AA@ 00409614     LIBCMT:crt0msg.obj
 0002:00000630       ??_C@_03KHICJKCI@?4?4?4?$AA@ 00409630     LIBCMT:crt0msg.obj
 0002:00000634       ??_C@_0BH@DNAGHKFM@?$DMprogram?5name?5unknown?$DO?$AA@ 00409634     LIBCMT:crt0msg.obj
 0002:0000064c       ??_C@_0CG@PKBDLMEO@InitializeCriticalSectionAndSpin@ 0040964c     LIBCMT:initcrit.obj
 0002:00000674       ??_C@_0N@MDJJJHMB@kernel32?4dll?$AA@ 00409674     LIBCMT:initcrit.obj
 0002:000006e4       ??_C@_13NOLLCAOD@?$AA?$AA?$AA?$AA@ 004096e4     LIBCMT:a_str.obj
 0002:000006f4       ??_C@_08JCCMCCIL@HH?3mm?3ss?$AA@ 004096f4     LIBCMT:strftime.obj
 0002:00000700       ??_C@_0BE@CKGJFCPC@dddd?0?5MMMM?5dd?0?5yyyy?$AA@ 00409700     LIBCMT:strftime.obj
 0002:00000714       ??_C@_08BPBNCDIB@MM?1dd?1yy?$AA@ 00409714     LIBCMT:strftime.obj
 0002:00000720       ??_C@_02CJNFDJBF@PM?$AA@   00409720     LIBCMT:strftime.obj
 0002:00000724       ??_C@_02DEDBPAFC@AM?$AA@   00409724     LIBCMT:strftime.obj
 0002:00000728       ??_C@_08EDHMEBNP@December?$AA@ 00409728     LIBCMT:strftime.obj
 0002:00000734       ??_C@_08HCHEGEOA@November?$AA@ 00409734     LIBCMT:strftime.obj
 0002:00000740       ??_C@_07JJNFCEND@October?$AA@ 00409740     LIBCMT:strftime.obj
 0002:00000748       ??_C@_09BHHEALKD@September?$AA@ 00409748     LIBCMT:strftime.obj
 0002:00000754       ??_C@_06LBBHFDDG@August?$AA@ 00409754     LIBCMT:strftime.obj
 0002:0000075c       ??_C@_04MIEPOIFP@July?$AA@ 0040975c     LIBCMT:strftime.obj
 0002:00000764       ??_C@_04CNLMGBGM@June?$AA@ 00409764     LIBCMT:strftime.obj
 0002:0000076c       ??_C@_05DMJDNLEJ@April?$AA@ 0040976c     LIBCMT:strftime.obj
 0002:00000774       ??_C@_05HPCKOFNC@March?$AA@ 00409774     LIBCMT:strftime.obj
 0002:0000077c       ??_C@_08GNJGEPFN@February?$AA@ 0040977c     LIBCMT:strftime.obj
 0002:00000788       ??_C@_07CGJPFGJA@January?$AA@ 00409788     LIBCMT:strftime.obj
 0002:00000790       ??_C@_03MKABNOCG@Dec?$AA@  00409790     LIBCMT:strftime.obj
 0002:00000794       ??_C@_03JPJOFNIA@Nov?$AA@  00409794     LIBCMT:strftime.obj
 0002:00000798       ??_C@_03BMAOKBAD@Oct?$AA@  00409798     LIBCMT:strftime.obj
 0002:0000079c       ??_C@_03GGCAPAJC@Sep?$AA@  0040979c     LIBCMT:strftime.obj
 0002:000007a0       ??_C@_03IFJFEIGA@Aug?$AA@  004097a0     LIBCMT:strftime.obj
 0002:000007a4       ??_C@_03LBGABGKK@Jul?$AA@  004097a4     LIBCMT:strftime.obj
 0002:000007a8       ??_C@_03IDFGHECI@Jun?$AA@  004097a8     LIBCMT:strftime.obj
 0002:000007ac       ??_C@_03CNMDKL@May?$AA@    004097ac     LIBCMT:strftime.obj
 0002:000007b0       ??_C@_03LEOLGMJP@Apr?$AA@  004097b0     LIBCMT:strftime.obj
 0002:000007b4       ??_C@_03ODNJBKGA@Mar?$AA@  004097b4     LIBCMT:strftime.obj
 0002:000007b8       ??_C@_03HJBDCHOM@Feb?$AA@  004097b8     LIBCMT:strftime.obj
 0002:000007bc       ??_C@_03JIHJHPIE@Jan?$AA@  004097bc     LIBCMT:strftime.obj
 0002:000007c0       ??_C@_08INBOOONO@Saturday?$AA@ 004097c0     LIBCMT:strftime.obj
 0002:000007cc       ??_C@_06JECMNKMI@Friday?$AA@ 004097cc     LIBCMT:strftime.obj
 0002:000007d4       ??_C@_08HACCIKIA@Thursday?$AA@ 004097d4     LIBCMT:strftime.obj
 0002:000007e0       ??_C@_09DLIGFAKA@Wednesday?$AA@ 004097e0     LIBCMT:strftime.obj
 0002:000007ec       ??_C@_07BAAGCFCM@Tuesday?$AA@ 004097ec     LIBCMT:strftime.obj
 0002:000007f4       ??_C@_06JLEDEDGH@Monday?$AA@ 004097f4     LIBCMT:strftime.obj
 0002:000007fc       ??_C@_06OOPIFAJ@Sunday?$AA@ 004097fc     LIBCMT:strftime.obj
 0002:00000804       ??_C@_03FEFJNEK@Sat?$AA@   00409804     LIBCMT:strftime.obj
 0002:00000808       ??_C@_03IDIOELNC@Fri?$AA@  00409808     LIBCMT:strftime.obj
 0002:0000080c       ??_C@_03IOFIKPDN@Thu?$AA@  0040980c     LIBCMT:strftime.obj
 0002:00000810       ??_C@_03MHOMLAJA@Wed?$AA@  00409810     LIBCMT:strftime.obj
 0002:00000814       ??_C@_03NAGEINEP@Tue?$AA@  00409814     LIBCMT:strftime.obj
 0002:00000818       ??_C@_03PDAGKDH@Mon?$AA@   00409818     LIBCMT:strftime.obj
 0002:0000081c       ??_C@_03KOEHGMDN@Sun?$AA@  0040981c     LIBCMT:strftime.obj
 0002:00000820       __ctype                    00409820     LIBCMT:ctype.obj
 0002:00000a28       __wctype                   00409a28     LIBCMT:ctype.obj
 0002:00000c94       ??_C@_0BI@DFKBFLJE@GetProcessWindowStation?$AA@ 00409c94     LIBCMT:crtmbox.obj
 0002:00000cac       ??_C@_0BK@CIDNPOGP@GetUserObjectInformationA?$AA@ 00409cac     LIBCMT:crtmbox.obj
 0002:00000cc8       ??_C@_0BD@HHGDFDBJ@GetLastActivePopup?$AA@ 00409cc8     LIBCMT:crtmbox.obj
 0002:00000cdc       ??_C@_0BA@HNOPNCHB@GetActiveWindow?$AA@ 00409cdc     LIBCMT:crtmbox.obj
 0002:00000cec       ??_C@_0M@CHKKJDAI@MessageBoxA?$AA@ 00409cec     LIBCMT:crtmbox.obj
 0002:00000cf8       ??_C@_0L@GMPLCCII@user32?4dll?$AA@ 00409cf8     LIBCMT:crtmbox.obj
 0002:00000d24       ___dnames                  00409d24     LIBCMT:timeset.obj
 0002:00000d3c       ___mnames                  00409d3c     LIBCMT:timeset.obj
 0002:00000d64       ??_C@_09KLGCKDOD@Program?3?5?$AA@ 00409d64     LIBCMT:secfail.obj
 0002:00000d70       ??_C@_0KA@JEHFIFGP@A?5buffer?5overrun?5has?5been?5detect@ 00409d70     LIBCMT:secfail.obj
 0002:00000e10       ??_C@_0BJ@MDEKIEOJ@Buffer?5overrun?5detected?$CB?$AA@ 00409e10     LIBCMT:secfail.obj
 0002:00000e30       ??_C@_0LB@BPLHHLFD@A?5security?5error?5of?5unknown?5caus@ 00409e30     LIBCMT:secfail.obj
 0002:00000ee4       ??_C@_0CD@GMKACBEK@Unknown?5security?5failure?5detecte@ 00409ee4     LIBCMT:secfail.obj
 0002:00000f24       ___rtc_iaa                 00409f24     LIBCMT:initsect.obj
 0002:00000f28       ___rtc_izz                 00409f28     LIBCMT:initsect.obj
 0002:00000f2c       ___rtc_taa                 00409f2c     LIBCMT:initsect.obj
 0002:00000f30       ___rtc_tzz                 00409f30     LIBCMT:initsect.obj
 0003:00000000       ___xc_a                    0040a000     LIBCMT:crt0init.obj
 0003:00000008       ___xc_z                    0040a008     LIBCMT:crt0init.obj
 0003:0000000c       ___xi_a                    0040a00c     LIBCMT:crt0init.obj
 0003:0000001c       ___xi_z                    0040a01c     LIBCMT:crt0init.obj
 0003:00000020       ___xp_a                    0040a020     LIBCMT:crt0init.obj
 0003:00000028       ___xp_z                    0040a028     LIBCMT:crt0init.obj
 0003:0000002c       ___xt_a                    0040a02c     LIBCMT:crt0init.obj
 0003:00000030       ___xt_z                    0040a030     LIBCMT:crt0init.obj
 0003:000011b0       __iob                      0040b1b0     LIBCMT:_file.obj
 0003:00001430       __aexit_rtn                0040b430     LIBCMT:crt0.obj
 0003:00001434       ___app_type                0040b434     LIBCMT:crt0.obj
 0003:00001438       ___badioinfo               0040b438     LIBCMT:ioinit.obj
 0003:00001588       ___initiallocinfo          0040b588     LIBCMT:setlocal.obj
 0003:000015dc       ___ptlocinfo               0040b5dc     LIBCMT:setlocal.obj
 0003:00001714       ___tlsindex                0040b714     LIBCMT:tidtable.obj
 0003:00001720       ___nullstring              0040b720     LIBCMT:output.obj
 0003:00001724       ___wnullstring             0040b724     LIBCMT:output.obj
 0003:000017c0       __XcptActTab               0040b7c0     LIBCMT:winxfltr.obj
 0003:00001838       __First_FPE_Indx           0040b838     LIBCMT:winxfltr.obj
 0003:0000183c       __Num_FPE                  0040b83c     LIBCMT:winxfltr.obj
 0003:00001840       __XcptActTabSize           0040b840     LIBCMT:winxfltr.obj
 0003:00001844       __XcptActTabCount          0040b844     LIBCMT:winxfltr.obj
 0003:00001848       __amblksiz                 0040b848     LIBCMT:heapinit.obj
 0003:000019b8       ___lc_time_curr            0040b9b8     LIBCMT:strftime.obj
 0003:000019c0       ___lc_time_c               0040b9c0     LIBCMT:strftime.obj
 0003:00001a78       __pctype                   0040ba78     LIBCMT:ctype.obj
 0003:00001a7c       __pwctype                  0040ba7c     LIBCMT:ctype.obj
 0003:00001a80       ___lconv_static_decimal    0040ba80     LIBCMT:lconv.obj
 0003:00001a84       ___lconv_c                 0040ba84     LIBCMT:lconv.obj
 0003:00001ab4       ___lconv                   0040bab4     LIBCMT:lconv.obj
 0003:00001ac0       ___security_cookie         0040bac0     LIBCMT:seccook.obj
 0003:00001ac4       ___lc_clike                0040bac4     LIBCMT:nlsdata2.obj
 0003:00001ad0       ___mb_cur_max              0040bad0     LIBCMT:nlsdata1.obj
 0003:00001ad4       ___decimal_point           0040bad4     LIBCMT:nlsdata1.obj
 0003:00001ad8       ___decimal_point_length    0040bad8     LIBCMT:nlsdata1.obj
 0003:00001adc       __NLG_Destination          0040badc     LIBCMT:exsup.obj
 0003:00001be8       __cfltcvt_tab              0040bbe8     LIBCMT:cmiscdat.obj
 0003:00001c00       __timezone                 0040bc00     LIBCMT:timeset.obj
 0003:00001c04       __daylight                 0040bc04     LIBCMT:timeset.obj
 0003:00001c08       __dstbias                  0040bc08     LIBCMT:timeset.obj
 0003:00001c90       __tzname                   0040bc90     LIBCMT:timeset.obj
 0003:00001cb0       __lpdays                   0040bcb0     LIBCMT:days.obj
 0003:00001ce4       __days                     0040bce4     LIBCMT:days.obj
 0003:00002c98       __cflush                   0040cc98     LIBCMT:_file.obj
 0003:00002c9c       __umaskval                 0040cc9c     LIBCMT:crt0dat.obj
 0003:00002ca0       __osplatform               0040cca0     LIBCMT:crt0dat.obj
 0003:00002ca4       __osver                    0040cca4     LIBCMT:crt0dat.obj
 0003:00002ca8       __winver                   0040cca8     LIBCMT:crt0dat.obj
 0003:00002cac       __winmajor                 0040ccac     LIBCMT:crt0dat.obj
 0003:00002cb0       __winminor                 0040ccb0     LIBCMT:crt0dat.obj
 0003:00002cb4       ___argc                    0040ccb4     LIBCMT:crt0dat.obj
 0003:00002cb8       ___argv                    0040ccb8     LIBCMT:crt0dat.obj
 0003:00002cbc       ___wargv                   0040ccbc     LIBCMT:crt0dat.obj
 0003:00002cc0       __environ                  0040ccc0     LIBCMT:crt0dat.obj
 0003:00002cc4       ___initenv                 0040ccc4     LIBCMT:crt0dat.obj
 0003:00002cc8       __wenviron                 0040ccc8     LIBCMT:crt0dat.obj
 0003:00002ccc       ___winitenv                0040cccc     LIBCMT:crt0dat.obj
 0003:00002cd0       __pgmptr                   0040ccd0     LIBCMT:crt0dat.obj
 0003:00002cd4       __wpgmptr                  0040ccd4     LIBCMT:crt0dat.obj
 0003:00002cd8       __exitflag                 0040ccd8     LIBCMT:crt0dat.obj
 0003:00002cdc       __C_Termination_Done       0040ccdc     LIBCMT:crt0dat.obj
 0003:00002ce0       __C_Exit_Done              0040cce0     LIBCMT:crt0dat.obj
 0003:00002ce4       __aenvptr                  0040cce4     LIBCMT:crt0.obj
 0003:00002ce8       __wenvptr                  0040cce8     LIBCMT:crt0.obj
 0003:00002cec       ___error_mode              0040ccec     LIBCMT:crt0.obj
 0003:00002e4c       __stdbuf                   0040ce4c     LIBCMT:_sftbuf.obj
 0003:00002e54       __adbgmsg                  0040ce54     LIBCMT:crt0msg.obj
 0003:00002f68       ?_pnhHeap@@3P6AHI@ZA       0040cf68     LIBCMT:handler.obj
 0003:00002f6c       __newmode                  0040cf6c     LIBCMT:_newmode.obj
 0003:00002f74       ___lconv_static_null       0040cf74     LIBCMT:lconv.obj
 0003:00002f78       ___lc_time_intl            0040cf78     LIBCMT:inittime.obj
 0003:00002f7c       ___lconv_intl              0040cf7c     LIBCMT:initmon.obj
 0003:00002fa4       ___lc_handle               0040cfa4     LIBCMT:nlsdata2.obj
 0003:00002fbc       ___lc_codepage             0040cfbc     LIBCMT:nlsdata2.obj
 0003:00002fc0       ___lc_collate_cp           0040cfc0     LIBCMT:nlsdata2.obj
 0003:00002fc4       ___lc_id                   0040cfc4     LIBCMT:nlsdata3.obj
 0003:000030d8       _verbose                   0040d0d8     <common>
 0003:000030dc       _progname                  0040d0dc     <common>
 0003:000030e0       ___mblcid                  0040d0e0     <common>
 0003:000030e4       ___ptmbcinfo               0040d0e4     <common>
 0003:000030e8       ___ismbcodepage            0040d0e8     <common>
 0003:00003100       __mbctype                  0040d100     <common>
 0003:00003204       ___mbcodepage              0040d204     <common>
 0003:00003210       ___mbulinfo                0040d210     <common>
 0003:00003220       __mbcasemap                0040d220     <common>
 0003:00003320       ___ctype1_refcount         0040d320     <common>
 0003:00003324       ___lconv_mon_refcount      0040d324     <common>
 0003:00003328       ___lconv_num_refcount      0040d328     <common>
 0003:0000332c       ___sbh_pHeaderDefer        0040d32c     <common>
 0003:00003330       ___sbh_cntHeaderList       0040d330     <common>
 0003:00003334       ___sbh_pHeaderList         0040d334     <common>
 0003:00003338       ___sbh_threshold           0040d338     <common>
 0003:0000333c       ___sbh_pHeaderScan         0040d33c     <common>
 0003:00003340       ___sbh_sizeHeaderList      0040d340     <common>
 0003:00003344       ___sbh_indGroupDefer       0040d344     <common>
 0003:00003348       __crtheap                  0040d348     <common>
 0003:0000334c       ___active_heap             0040d34c     <common>
 0003:00003350       __nhandle                  0040d350     <common>
 0003:00003360       ___pioinfo                 0040d360     <common>
 0003:00003460       __acmdln                   0040d460     <common>
 0003:00003464       ___env_initialized         0040d464     <common>
 0003:00003468       ___onexitend               0040d468     <common>
 0003:0000346c       ___onexitbegin             0040d46c     <common>
 0003:00003470       ___mbctype_initialized     0040d470     <common>
 0003:00003474       __FPinit                   0040d474     <common>
 0003:00003478       ___piob                    0040d478     <common>
 0003:00003480       __bufin                    0040d480     <common>
 0003:00004480       __nstream                  0040e480     <common>
 0004:00000000       __IMPORT_DESCRIPTOR_libisc 0040f000     libisc:libisc.dll
 0004:00000014       __IMPORT_DESCRIPTOR_libisccfg 0040f014     libisccfg:libisccfg.dll
 0004:00000028       __IMPORT_DESCRIPTOR_libisccc 0040f028     libisccc:libisccc.dll
 0004:0000003c       __IMPORT_DESCRIPTOR_libbind9 0040f03c     libbind9:libbind9.dll
 0004:00000050       __IMPORT_DESCRIPTOR_KERNEL32 0040f050     kernel32:KERNEL32.dll
 0004:00000064       __NULL_IMPORT_DESCRIPTOR   0040f064     libisc:libisc.dll
 0004:000002ac       __imp__MultiByteToWideChar@24 0040f2ac     kernel32:KERNEL32.dll
 0004:000002b0       __imp__GetStringTypeA@20   0040f2b0     kernel32:KERNEL32.dll
 0004:000002b4       __imp__FlushFileBuffers@4  0040f2b4     kernel32:KERNEL32.dll
 0004:000002b8       __imp__HeapReAlloc@16      0040f2b8     kernel32:KERNEL32.dll
 0004:000002bc       __imp__VirtualAlloc@16     0040f2bc     kernel32:KERNEL32.dll
 0004:000002c0       __imp__InitializeCriticalSection@4 0040f2c0     kernel32:KERNEL32.dll
 0004:000002c4       __imp__HeapFree@12         0040f2c4     kernel32:KERNEL32.dll
 0004:000002c8       __imp__VirtualFree@12      0040f2c8     kernel32:KERNEL32.dll
 0004:000002cc       __imp__HeapCreate@12       0040f2cc     kernel32:KERNEL32.dll
 0004:000002d0       __imp__HeapDestroy@4       0040f2d0     kernel32:KERNEL32.dll
 0004:000002d4       __imp__GetEnvironmentStringsW@0 0040f2d4     kernel32:KERNEL32.dll
 0004:000002d8       __imp__WideCharToMultiByte@32 0040f2d8     kernel32:KERNEL32.dll
 0004:000002dc       __imp__FreeEnvironmentStringsW@4 0040f2dc     kernel32:KERNEL32.dll
 0004:000002e0       __imp__GetEnvironmentStrings@0 0040f2e0     kernel32:KERNEL32.dll
 0004:000002e4       __imp__FreeEnvironmentStringsA@4 0040f2e4     kernel32:KERNEL32.dll
 0004:000002e8       __imp__UnhandledExceptionFilter@4 0040f2e8     kernel32:KERNEL32.dll
 0004:000002ec       __imp__GetModuleFileNameA@12 0040f2ec     kernel32:KERNEL32.dll
 0004:000002f0       __imp__WriteFile@20        0040f2f0     kernel32:KERNEL32.dll
 0004:000002f4       __imp__TlsAlloc@0          0040f2f4     kernel32:KERNEL32.dll
 0004:000002f8       __imp__GetLastError@0      0040f2f8     kernel32:KERNEL32.dll
 0004:000002fc       __imp__TlsGetValue@4       0040f2fc     kernel32:KERNEL32.dll
 0004:00000300       __imp__TlsSetValue@8       0040f300     kernel32:KERNEL32.dll
 0004:00000304       __imp__GetCurrentThreadId@0 0040f304     kernel32:KERNEL32.dll
 0004:00000308       __imp__SetLastError@4      0040f308     kernel32:KERNEL32.dll
 0004:0000030c       __imp__TlsFree@4           0040f30c     kernel32:KERNEL32.dll
 0004:00000310       __imp__HeapAlloc@12        0040f310     kernel32:KERNEL32.dll
 0004:00000314       __imp__DeleteCriticalSection@4 0040f314     kernel32:KERNEL32.dll
 0004:00000318       __imp__GetStartupInfoA@4   0040f318     kernel32:KERNEL32.dll
 0004:0000031c       __imp__GetFileType@4       0040f31c     kernel32:KERNEL32.dll
 0004:00000320       __imp__GetStdHandle@4      0040f320     kernel32:KERNEL32.dll
 0004:00000324       __imp__SetHandleCount@4    0040f324     kernel32:KERNEL32.dll
 0004:00000328       __imp__GetVersionExA@4     0040f328     kernel32:KERNEL32.dll
 0004:0000032c       __imp__GetCommandLineA@0   0040f32c     kernel32:KERNEL32.dll
 0004:00000330       __imp__GetCurrentProcess@0 0040f330     kernel32:KERNEL32.dll
 0004:00000334       __imp__TerminateProcess@8  0040f334     kernel32:KERNEL32.dll
 0004:00000338       __imp__GetModuleHandleA@4  0040f338     kernel32:KERNEL32.dll
 0004:0000033c       __imp__GetProcAddress@8    0040f33c     kernel32:KERNEL32.dll
 0004:00000340       __imp__ExitProcess@4       0040f340     kernel32:KERNEL32.dll
 0004:00000344       __imp__LeaveCriticalSection@4 0040f344     kernel32:KERNEL32.dll
 0004:00000348       __imp__EnterCriticalSection@4 0040f348     kernel32:KERNEL32.dll
 0004:0000034c       __imp__GetCPInfo@8         0040f34c     kernel32:KERNEL32.dll
 0004:00000350       __imp__GetSystemTimeAsFileTime@4 0040f350     kernel32:KERNEL32.dll
 0004:00000354       __imp__GetCurrentProcessId@0 0040f354     kernel32:KERNEL32.dll
 0004:00000358       __imp__GetTickCount@0      0040f358     kernel32:KERNEL32.dll
 0004:0000035c       __imp__QueryPerformanceCounter@4 0040f35c     kernel32:KERNEL32.dll
 0004:00000360       __imp__VirtualQuery@12     0040f360     kernel32:KERNEL32.dll
 0004:00000364       __imp__GetSystemInfo@4     0040f364     kernel32:KERNEL32.dll
 0004:00000368       __imp__VirtualProtect@16   0040f368     kernel32:KERNEL32.dll
 0004:0000036c       __imp__SetStdHandle@8      0040f36c     kernel32:KERNEL32.dll
 0004:00000370       __imp__SetFilePointer@16   0040f370     kernel32:KERNEL32.dll
 0004:00000374       __imp__CloseHandle@4       0040f374     kernel32:KERNEL32.dll
 0004:00000378       __imp__LoadLibraryA@4      0040f378     kernel32:KERNEL32.dll
 0004:0000037c       __imp__LCMapStringW@24     0040f37c     kernel32:KERNEL32.dll
 0004:00000380       __imp__LCMapStringA@24     0040f380     kernel32:KERNEL32.dll
 0004:00000384       __imp__HeapSize@12         0040f384     kernel32:KERNEL32.dll
 0004:00000388       __imp__GetOEMCP@0          0040f388     kernel32:KERNEL32.dll
 0004:0000038c       __imp__GetACP@0            0040f38c     kernel32:KERNEL32.dll
 0004:00000390       __imp__RtlUnwind@16        0040f390     kernel32:KERNEL32.dll
 0004:00000394       __imp__GetLocaleInfoA@16   0040f394     kernel32:KERNEL32.dll
 0004:00000398       __imp__GetStringTypeW@16   0040f398     kernel32:KERNEL32.dll
 0004:0000039c       \177KERNEL32_NULL_THUNK_DATA 0040f39c     kernel32:KERNEL32.dll
 0004:000003a0       __imp__bind9_getaddresses  0040f3a0     libbind9:libbind9.dll
 0004:000003a4       \177libbind9_NULL_THUNK_DATA 0040f3a4     libbind9:libbind9.dll
 0004:000003a8       __imp__isc_mem_destroy     0040f3a8     libisc:libisc.dll
 0004:000003ac       __imp__isc_task_shutdown   0040f3ac     libisc:libisc.dll
 0004:000003b0       __imp__isc_file_exists     0040f3b0     libisc:libisc.dll
 0004:000003b4       __imp__isc_app_shutdown    0040f3b4     libisc:libisc.dll
 0004:000003b8       __imp__isc_error_runtimecheck 0040f3b8     libisc:libisc.dll
 0004:000003bc       __imp__isc_socket_detach   0040f3bc     libisc:libisc.dll
 0004:000003c0       __imp__isc_stdtime_get     0040f3c0     libisc:libisc.dll
 0004:000003c4       __imp__isc__buffer_init    0040f3c4     libisc:libisc.dll
 0004:000003c8       __imp__isc__buffer_putuint32 0040f3c8     libisc:libisc.dll
 0004:000003cc       __imp__isc_socket_send     0040f3cc     libisc:libisc.dll
 0004:000003d0       __imp__isc_sockaddr_format 0040f3d0     libisc:libisc.dll
 0004:000003d4       __imp__isc_sockaddr_pf     0040f3d4     libisc:libisc.dll
 0004:000003d8       __imp__isc_socket_create   0040f3d8     libisc:libisc.dll
 0004:000003dc       __imp__isc_socket_connect  0040f3dc     libisc:libisc.dll
 0004:000003e0       __imp__isc_app_block       0040f3e0     libisc:libisc.dll
 0004:000003e4       __imp__isc_app_unblock     0040f3e4     libisc:libisc.dll
 0004:000003e8       __imp__isc_event_free      0040f3e8     libisc:libisc.dll
 0004:000003ec       __imp__isc_file_progname   0040f3ec     libisc:libisc.dll
 0004:000003f0       __imp__isc_ntpaths_get     0040f3f0     libisc:libisc.dll
 0004:000003f4       __imp__isc_app_start       0040f3f4     libisc:libisc.dll
 0004:000003f8       __imp__isc_result_totext   0040f3f8     libisc:libisc.dll
 0004:000003fc       __imp__isc_commandline_parse 0040f3fc     libisc:libisc.dll
 0004:00000400       __imp__isc_commandline_argument 0040f400     libisc:libisc.dll
 0004:00000404       __imp__isc_mem_debugging   0040f404     libisc:libisc.dll
 0004:00000408       __imp__isc_commandline_index 0040f408     libisc:libisc.dll
 0004:0000040c       __imp__isc_random_get      0040f40c     libisc:libisc.dll
 0004:00000410       __imp__isc_mem_create      0040f410     libisc:libisc.dll
 0004:00000414       __imp__isc_socketmgr_create 0040f414     libisc:libisc.dll
 0004:00000418       __imp__isc_taskmgr_create  0040f418     libisc:libisc.dll
 0004:0000041c       __imp__isc_task_create     0040f41c     libisc:libisc.dll
 0004:00000420       __imp__isc_log_create      0040f420     libisc:libisc.dll
 0004:00000424       __imp__isc_log_setcontext  0040f424     libisc:libisc.dll
 0004:00000428       __imp__isc_log_settag      0040f428     libisc:libisc.dll
 0004:0000042c       __imp__isc_log_createchannel 0040f42c     libisc:libisc.dll
 0004:00000430       __imp__isc_log_usechannel  0040f430     libisc:libisc.dll
 0004:00000434       __imp__isc__mem_get        0040f434     libisc:libisc.dll
 0004:00000438       __imp__isc_assertion_failed 0040f438     libisc:libisc.dll
 0004:0000043c       __imp__isc_app_onrun       0040f43c     libisc:libisc.dll
 0004:00000440       __imp__isc_app_run         0040f440     libisc:libisc.dll
 0004:00000444       __imp__isc_socket_cancel   0040f444     libisc:libisc.dll
 0004:00000448       __imp__isc_task_detach     0040f448     libisc:libisc.dll
 0004:0000044c       __imp__isc_taskmgr_destroy 0040f44c     libisc:libisc.dll
 0004:00000450       __imp__isc_socketmgr_destroy 0040f450     libisc:libisc.dll
 0004:00000454       __imp__isc_log_destroy     0040f454     libisc:libisc.dll
 0004:00000458       __imp__isc__mem_put        0040f458     libisc:libisc.dll
 0004:0000045c       __imp__isc_mem_stats       0040f45c     libisc:libisc.dll
 0004:00000460       \177libisc_NULL_THUNK_DATA 0040f460     libisc:libisc.dll
 0004:00000464       __imp__isccc_base64_decode 0040f464     libisccc:libisccc.dll
 0004:00000468       __imp__isccc_cc_lookupstring 0040f468     libisccc:libisccc.dll
 0004:0000046c       __imp__isccc_cc_fromwire   0040f46c     libisccc:libisccc.dll
 0004:00000470       __imp__isccc_cc_lookupuint32 0040f470     libisccc:libisccc.dll
 0004:00000474       __imp__isccc_cc_defineuint32 0040f474     libisccc:libisccc.dll
 0004:00000478       __imp__isccc_ccmsg_cancelread 0040f478     libisccc:libisccc.dll
 0004:0000047c       __imp__isccc_sexpr_free    0040f47c     libisccc:libisccc.dll
 0004:00000480       __imp__isccc_cc_createmessage 0040f480     libisccc:libisccc.dll
 0004:00000484       __imp__isccc_alist_lookup  0040f484     libisccc:libisccc.dll
 0004:00000488       __imp__isccc_cc_definestring 0040f488     libisccc:libisccc.dll
 0004:0000048c       __imp__isccc_cc_towire     0040f48c     libisccc:libisccc.dll
 0004:00000490       __imp__isccc_ccmsg_init    0040f490     libisccc:libisccc.dll
 0004:00000494       __imp__isccc_ccmsg_setmaxsize 0040f494     libisccc:libisccc.dll
 0004:00000498       __imp__isccc_ccmsg_readmessage 0040f498     libisccc:libisccc.dll
 0004:0000049c       __imp__isccc_result_register 0040f49c     libisccc:libisccc.dll
 0004:000004a0       __imp__isccc_ccmsg_invalidate 0040f4a0     libisccc:libisccc.dll
 0004:000004a4       \177libisccc_NULL_THUNK_DATA 0040f4a4     libisccc:libisccc.dll
 0004:000004a8       __imp__cfg_type_rndcconf   0040f4a8     libisccfg:libisccfg.dll
 0004:000004ac       __imp__cfg_type_rndckey    0040f4ac     libisccfg:libisccfg.dll
 0004:000004b0       __imp__cfg_parser_create   0040f4b0     libisccfg:libisccfg.dll
 0004:000004b4       __imp__cfg_parse_file      0040f4b4     libisccfg:libisccfg.dll
 0004:000004b8       __imp__cfg_map_get         0040f4b8     libisccfg:libisccfg.dll
 0004:000004bc       __imp__cfg_obj_asstring    0040f4bc     libisccfg:libisccfg.dll
 0004:000004c0       __imp__cfg_list_first      0040f4c0     libisccfg:libisccfg.dll
 0004:000004c4       __imp__cfg_list_next       0040f4c4     libisccfg:libisccfg.dll
 0004:000004c8       __imp__cfg_listelt_value   0040f4c8     libisccfg:libisccfg.dll
 0004:000004cc       __imp__cfg_map_getname     0040f4cc     libisccfg:libisccfg.dll
 0004:000004d0       __imp__cfg_obj_asuint32    0040f4d0     libisccfg:libisccfg.dll
 0004:000004d4       __imp__cfg_obj_destroy     0040f4d4     libisccfg:libisccfg.dll
 0004:000004d8       __imp__cfg_parser_destroy  0040f4d8     libisccfg:libisccfg.dll
 0004:000004dc       \177libisccfg_NULL_THUNK_DATA 0040f4dc     libisccfg:libisccfg.dll

 entry point at        0001:0000247b

 Static symbols

 0001:000007bd       _usage                     004017bd f   rndc.obj
 0001:000007e8       _rndc_start                004017e8 f   rndc.obj
 0001:0000083b       _get_addresses             0040183b f   rndc.obj
 0001:000008af       _rndc_startconnect         004018af f   rndc.obj
 0001:000009a0       _rndc_connected            004019a0 f   rndc.obj
 0001:00000cab       _rndc_senddone             00401cab f   rndc.obj
 0001:00000cee       _rndc_recvnonce            00401cee f   rndc.obj
 0001:00001079       _rndc_recvdone             00402079 f   rndc.obj
 0001:0000126a       _parse_config              0040226a f   rndc.obj
 0001:00007b40       _$$$00001                  00408b40 f   LIBCMT:strchr.obj
 0001:00003200       _write_char                00404200 f   LIBCMT:output.obj
 0001:00003233       _write_multi_char          00404233 f   LIBCMT:output.obj
 0001:00003257       _write_string              00404257 f   LIBCMT:output.obj
 0001:00002a17       _flsall                    00403a17 f   LIBCMT:fflush.obj
 0001:00004070       _parse_cmdline             00405070 f   LIBCMT:stdargv.obj
 0001:00002124       _doexit                    00403124 f   LIBCMT:crt0dat.obj
 0001:00002457       _fast_error_exit           00403457 f   LIBCMT:crt0.obj
 0001:00002d99       ___updatetlocinfo_lk       00403d99 f   LIBCMT:setlocal.obj
 0001:00002fd4       __onexit_lk                00403fd4 f   LIBCMT:onexit.obj
 0001:0000444d       ___crtInitCritSecNoSpinCount@8 0040544d f   LIBCMT:initcrit.obj
 0001:00005ce4       _report_failure            00406ce4 f   LIBCMT:seccook.obj
 0001:000069b8       $$$00003                   004079b8 f   LIBCMT:exsup3.obj
 0001:00005e70       $$$00001                   00406e70 f   LIBCMT:exsup.obj
 0001:00005e90       $$$00003                   00406e90 f   LIBCMT:exsup.obj
 0001:00005e90       __unwind_handler           00406e90 f   LIBCMT:exsup.obj
 0001:00005eb2       $$$00005                   00406eb2 f   LIBCMT:exsup.obj
 0001:00005f1a       $$$00007                   00406f1a f   LIBCMT:exsup.obj
 0001:00005f5e       $$$00011                   00406f5e f   LIBCMT:exsup.obj
 0001:00005f5e       _CPtoLCID                  00406f5e f   LIBCMT:mbctype.obj
 0001:00005f8d       _setSBCS                   00406f8d f   LIBCMT:mbctype.obj
 0001:00005fb6       _setSBUpLow                00406fb6 f   LIBCMT:mbctype.obj
 0001:00006148       __setmbcp_lk               00407148 f   LIBCMT:mbctype.obj
